:020000040000FA
:100000009D280F39A0000310A00DA00D1F08E03996
:10001000200401389F000030A100323039209F14A5
:100020009F1810281E08A10083161E089828831602
:100030001C141A0883169B0A9828030183169A0039
:100040001C1555309D00AA309D009C149C18262834
:100050001C119B0A9828A301A200FF30A207031CD1
:10006000A307031C98280330A100DF3039202D2876
:10007000A101E83EA000A109FC30031C4228A00712
:1000800003183F28A0076400A10F3F282018482824
:10009000A01C4C2800004C280800A701A6001C301A
:1000A000A2006F30A30082200F30831681048312D8
:1000B000FF306300A007031CA107031859289828E4
:1000C0000310A10CA00CFF3E0318602820089828FC
:1000D000A20003307228A301A20001307228A200FE
:1000E00006307228A80023082102031D792822085F
:1000F0002002043003180130031902302805031DC3
:10010000FF3098281030A800A101A001A70CA60C70
:10011000031C90282208A00723080318230FA10717
:10012000A10CA00CA50CA40CA80B862824089828C8
:10013000831303138312640008009F17831608308B
:100140009F008312073099008316851683120330AF
:10015000A300E8302C206400851AAF284C298316B0
:100160009B0183121720D100831601309B0083125C
:100170001720D000CA01CB014A08A0004B08A100FB
:10018000A30107306C20031DFE2803300120C800A6
:100190002108C9000330A300E8302C20510848078B
:1001A000CC0049080318013ECD0050084C02C8009D
:1001B0004D08031CFF3EC9004808A6004908A700D7
:1001C000C830A200A30182202508CC002008CD0061
:1001D0004C08A0004D08A10002306320C80021088F
:1001E000C90003104A0D383E840048088000840A84
:1001F00049088000CA0A0319CB0FBC281F223C08FB
:100200003E07CC003D080318013E3F07CD004008E3
:10021000CC0741080318013ECD074208CC0743082C
:100220000318013ECD074C08A0004D08A100023084
:100230006320C8002108C900851483168510831225
:100240000330A300E8302C2085108316851083121C
:100250000130CA00CB014A08A0004B08A1004908A0
:10026000A30048086C20031D4729051083160510BC
:1002700083120130A3002C302C20051483160510A6
:10028000143083122B20CA0A0319CB0F2B293C30C0
:100290004D20BA2863004A290130CA00CB014A0820
:1002A000A0004B08A100A30103306C20031D6C29A2
:1002B00085148316851083120230A30058302C2039
:1002C00085108316851083120330A30084302C2000
:1002D000CA0A0319CB0F4F29D101D001CA01CB01A2
:1002E0004A08A0004B08A100A30107306C20031DA1
:1002F0008D2903300120C8002108C90064302B205B
:1003000003104A0D383E840048088000840A4908DA
:100310008000CA0A0319CB0F70291F223C083E0730
:10032000CC003D080318013E3F07CD004008CC0734
:1003300041080318013ECD074208CC0743080318C3
:10034000013ECD074C08A0004D08A10002306320FB
:10035000C8002108C9004808A0004908A1000230CF
:10036000A30066306F20031DB92966304802D10012
:10037000D0014808A0004908A1000230A30066305F
:100380006820031DC729D1014808663CD0008316A8
:100390009B01831251081E20831601309B0083129B
:1003A00050081E206400500851020318D929500833
:1003B000D1000130CA00CB014A08A0004B08A100BF
:1003C00051086B20031DF6290510831605108312B2
:1003D0000130A3002C302C20051483160510143096
:1003E00083122B20CA0A0319CB0FDC290330A30088
:1003F000E8302C200130CA00CB014A08A0004B088D
:10040000A100A30105306C20031D1A2A8514831650
:10041000851083120230A30058302C2085108316DB
:10042000851083120330A30084302C20CA0A0319DC
:10043000CB0FFD292730A30010302C204C29CA01F6
:10044000CB0101304A07CC004B080318013ECD0018
:1004500003104C0D383E84000008CC00840A0008CC
:10046000CD0003104A0D383E84000008CE00840AF7
:100470000008CF004C08A0004D08A1004F08A300C1
:100480004E086820031D892A03104A0D383E840057
:100490000008C800840A0008C90001304A07CC00DF
:1004A0004B080318013ECD0003104C0D383E84006C
:1004B0000008CC00840A0008CD0003104A0D383E25
:1004C00084004C088000840A4D08800001304A07EF
:1004D000CC004B080318013ECD000030CC070318B8
:1004E000CD0A03104C0D383E840048088000840A71
:1004F000490880004A08A0004B08A100A301003071
:100500006F20031D892A0230CA020030031C013EFD
:10051000CB02CA0A0319CB0A4A08A0004B08A10063
:0E052000A30107306820031D962A212A080037
:02400E00FC3F75
:0442000000000000BA
:00000001FF
